:020000040000FA
:0600000052EF07F01200B0
:0608000052EF07F01200A8
:06082A000100C20E0000F7
:0808300000020000300000008E
:08083800D9CFE6FFE1CFD9FFA3
:10084000040EE126DE6ADE6ADE6ADD6ADD52DD5212
:10085000FD0EDBCF00F0FE0EDBCF01F0026A036A73
:1008600001AE02D002680368D9CFE9FFDACFEAFF10
:10087000030EEB500318E8AE02D0033408D000504A
:10088000EE5C0150EE580250EE580350EE580FE265
:100890000C0EE66E32EC07F0E552D9CFE9FFDACF65
:1008A000EAFFEE2A000EEE22EE22EE22D1D7040E4F
:1008B000E15C02E2E16AE552E16EE552E7CFD9FF81
:1008C00012000F0EC16E070EB46E936A300E926E58
:1008D0000F0E946EF19E1200D9CFE6FFE1CFD9FF43
:1008E000020EE1268250020B01E0010E080DF3CF4B
:1008F00002F08250010B040DF3CF01F08050200B69
:1009000001E0010EE824006E8050100B01E0010EA2
:10091000002401240224DE6EDD6ADECF00F0DDCF8C
:1009200001F000C0F3FF01C0F4FF020EE15C03E23E
:1009300000D0E16AE552E16EE552E7CFD9FF12003F
:100940008092010EE66EE66A77DFE552E55280841A
:10095000010EE66EE66A70DFE552E5528094010E04
:10096000E66EE66A69DFE552E55212008082010E0A
:10097000E66EE66A61DFE552E5528084010EE66EBE
:10098000E66A5ADFE552E5528094010EE66EE66AA9
:1009900053DFE552E5521200380E816ED1DF320E80
:1009A000E66EE66A49DFE552E552010E816EC8DF68
:1009B000320EE66EE66A40DFE552E5520D0E816EBC
:1009C000BFDF320EE66EE66A37DFE552E552060E0D
:1009D000816EB6DF320EE66EE66A2EDFE552E55234
:1009E0001200010E816EACDF0A0EE66EE66A24DFAD
:1009F000E552E5521200D9CFE6FFE1CFD9FF020E52
:100A0000816E9EDF0A0EE66EE66A16DFE552E5525B
:100A1000FD0EDBCFE6FFFE0EDB50280DF350E55256
:100A2000E724E76EFE0EE7CFDBFFFD0EDB6AFE0E6E
:100A3000DB50F36EFD0EDBCFF4FFF350F45C0CE201
:100A4000140E816E7DDF010EE66EE66AF5DEE5527C
:100A5000E552FD0EDB2AEBD7E552E7CFD9FF1200B6
:100A6000D9CFE6FFE1CFD9FFFE0EDB50816E7EDFEE
:100A7000010EE66EE66AE0DEE552E552E552E7CFAA
:100A8000D9FF1200D9CFE6FFE1CFD9FFFD0EDBCFB2
:100A9000E9FFFE0EDBCFEAFFEF500EE0FD0EDBCFED
:100AA000E9FFDB2AFE0EDBCFEAFF01E3DB2AEF5092
:100AB000E66ED6DFE552EAD7E552E7CFD9FF12005E
:100AC0000001646B300E926EF00E936EEF0E606F4D
:100AD00060C081FF040E616F6151000821E2605126
:100AE000FE0BE842606F60C081FF050EE66EE66AAD
:100AF000A3DEE552E5528150100B09E08150200B36
:100B000006E08150400B03E08150800B01E10AD8E0
:100B10000001640502E1655104D06105616FDCD715
:100B2000CFD71200F00E936E81CF63F000016315F2
:100B3000626F0F0E6015606F60516211606F81CF40
:100B400063F0F00E6315626FF00E625D01E0F7D79F
:100B5000936A06D866C065F00001010E646F12004A
:100B60000001676B100E675D14E26751EA6A000FBF
:100B7000E96E020EEA22EF50605D08E16751EA6A11
:100B8000100FE96E020EEA22EFCF66F06729676F59
:100B9000E9D766C081FF640EE66EE66A4DDEE55277
:100BA000E55212000001686B070E685D1DE288DFE8
:100BB0000001696F6851EA6A6A0FE96E000EEA2265
:100BC00069C0EFFF6851EA6A6A0FE96E000EEA2217
:100BD000EF50460802E108D004D069C0E6FF40DFCC
:100BE000E5520001682BE0D76851EA6A6A0FE96EA6
:100BF000000EEA22EF6A12000001686B070E685DC2
:100C000016E26851EA6A6A0FE96E000EEA22EF50B6
:100C1000E66E26DFE55200016829EA6A6A0FE96E8E
:100C2000000EEA22EF5001E102D0682BE7D7120054
:100C300048DEB2DED6DEE66AE66ADDDEE552E55281
:100C4000200EE66E020EE66E1DDFE552E552E66A04
:100C5000010EE66ED0DEE552E552A4DF6A0EE66EC6
:100C6000000EE66E6EEC06F0E552E552F3CF73F03F
:100C7000F4CF74F00001756B766B74AF02D07569B8
:100C80007669500E731906E10D0E741903E1755162
:100C900001E1765112E1A5DE280EE66E020EE66E47
:100CA000F1DEE552E5528080D00EE66E070EE66E6C
:100CB000C3DDE552E55280900FD093DE2D0EE66E37
:100CC000020EE66EDFDEE552E552E80EE66E030E3A
:0C0CD000E66EB2DDE552E552ADD7120031
:040CDC00FF0EE3CF55
:100CE000EAFFE552FF0EE3CFE9FFE552E66AE66A66
:100CF000D9CFE6FFDACFE6FFFC0EE124D96EFF0E76
:100D0000E220DA6EE66AE66AE66A200EEF5C06E04A
:100D1000090EEF5C03E0EF6603D03FD0EE50F5D74D
:100D20002D0EEF5C03E1FF0EE32A03D02B0EEF5CE8
:100D300001E1EE502F0EEF6424D03A0EEF6021D087
:100D4000D890F90EE336FA0EE336FD0EDECFE3FF60
:100D5000FE0EDDCFE3FFD890F90EE336FA0EE33650
:100D6000D890F90EE336FA0EE336FD0EE350DE2698
:100D7000FE0EE350DD22300EEE5CDE26000EDD229C
:100D8000D9D7FF0EE3CFE8FFE85207E0F90EE31EE4
:100D9000E32AFA0ED8B4E306E31EE552E552E55223
:100DA000FF0EE3CFDAFFE552FF0EE3CFD9FFE552A6
:100DB000E1CFE9FFE2CFEAFFED52ED52EECFF3FFD4
:060DC000EFCFF4FF12006A
:0A0DC6002A0EF66E080EF76E000EFE
:100DD000F86E02010900F550356F0900F550366FC5
:100DE00003E1356701D03DD00900F550306F0900AF
:100DF000F550316F0900F550326F09000900F550C8
:100E0000E96E0900F550EA6E090009000900F55085
:100E1000336F0900F550346F09000900F6CF37F23F
:100E2000F7CF38F2F8CF39F230C2F6FF31C2F7FF10
:100E300032C2F8FF0201335302E1345307E00900E4
:100E4000F550EE6E3307F8E23407F9D737C2F6FFF4
:100E500038C2F7FF39C2F8FF02013507000E365BD2
:040E6000BFD71200E6
:0C0E6400FF0EE350066E480E01D04C0E4D
:100E7000E76EE72EFED7E76AE72EFED7062EF7D7F6
:040E8000000012005C
:0C0E8400000EF36E00EE00F0080E01D826
:100E90001200EA6002D0EE6AFCD7F350E96012005B
:040EA000EE6AFCD723
:0C0EA40012EE40F022EE40F0F86A059CCF
:100EB000E3EC06F060EC07F018EC06F0FBD712004C
:020EC00012001E
:0E0EC200EEEDEBE7DEDDDBD7BEBDBBB77E7D20
:100ED0007B77303132333435363738394142434409
:100EE0004546434C4156453E3E004F4B2121006E46
:020EF0006F0091
:00000001FF
